ARM Linker, RVCT3.1 [Build 914] for uVision [Standard]

================================================================================

Section Cross References

    startup.o(STACK) refers (Special) to stkheap2.o(.text) for __use_two_region_memory
    startup.o(HEAP) refers (Special) to stkheap2.o(.text) for __use_two_region_memory
    startup.o(RESET) refers to startup.o(STACK) for StackMem
    startup.o(RESET) refers to uart_echo.o(.text) for UARTIntHandler
    startup.o(RESET) refers to __main.o(!!!main) for __main
    startup.o(RESET) refers (Special) to stkheap2.o(.text) for __use_two_region_memory
    startup.o(.text) refers to startup.o(HEAP) for HeapMem
    startup.o(.text) refers to startup.o(STACK) for StackMem
    startup.o(.text) refers (Special) to stkheap2.o(.text) for __use_two_region_memory
    pcd5544.o(.text) refers to sysctl.o(i.SysCtlPeripheralEnable) for SysCtlPeripheralEnable
    pcd5544.o(.text) refers to timer.o(i.TimerConfigure) for TimerConfigure
    pcd5544.o(.text) refers to timer.o(i.TimerLoadSet) for TimerLoadSet
    pcd5544.o(.text) refers to gpio.o(i.GPIODirModeSet) for GPIODirModeSet
    pcd5544.o(.text) refers to timer.o(i.TimerMatchSet) for TimerMatchSet
    pcd5544.o(.text) refers to timer.o(i.TimerEnable) for TimerEnable
    pcd5544.o(.text) refers to timer.o(i.TimerDisable) for TimerDisable
    pcd5544.o(.text) refers to gpio.o(i.GPIOPinWrite) for GPIOPinWrite
    pcd5544.o(.text) refers to gpio.o(i.GPIOPadConfigSet) for GPIOPadConfigSet
    pcd5544.o(.text) refers to ssi.o(i.SSIConfig) for SSIConfig
    pcd5544.o(.text) refers to ssi.o(i.SSIEnable) for SSIEnable
    pcd5544.o(.text) refers to ssi.o(i.SSIDataPut) for SSIDataPut
    pcd5544.o(.text) refers to pcd5544.o(.constdata) for ASC2
    uart_echo.o(.text) refers to uart.o(.text) for UARTIntStatus
    uart_echo.o(.text) refers to sysctl.o(i.SysCtlClockSet) for SysCtlClockSet
    uart_echo.o(.text) refers to sysctl.o(i.SysCtlPeripheralEnable) for SysCtlPeripheralEnable
    uart_echo.o(.text) refers to gpio.o(i.GPIODirModeSet) for GPIODirModeSet
    uart_echo.o(.text) refers to gpio.o(i.GPIOPadConfigSet) for GPIOPadConfigSet
    uart_echo.o(.text) refers to gpio.o(i.GPIOPinRead) for GPIOPinRead
    uart_echo.o(.text) refers to pcd5544.o(.text) for LCD_Backlight_On
    uart_echo.o(.text) refers to interrupt.o(i.IntMasterEnable) for IntMasterEnable
    uart_echo.o(.text) refers to gpio.o(i.GPIOPinTypeUART) for GPIOPinTypeUART
    uart_echo.o(.text) refers to sysctl.o(i.SysCtlClockGet) for SysCtlClockGet
    uart_echo.o(.text) refers to interrupt.o(i.IntEnable) for IntEnable
    uart_echo.o(.text) refers to gpio.o(i.GPIOPinWrite) for GPIOPinWrite
    uart.o(.text) refers to interrupt.o(i.IntRegister) for IntRegister
    uart.o(.text) refers to interrupt.o(i.IntEnable) for IntEnable
    uart.o(.text) refers to interrupt.o(i.IntDisable) for IntDisable
    uart.o(.text) refers to interrupt.o(i.IntUnregister) for IntUnregister
    gpio.o(i.GPIOPortIntRegister) refers to gpio.o(i.GPIOGetIntNumber) for GPIOGetIntNumber
    gpio.o(i.GPIOPortIntRegister) refers to interrupt.o(i.IntRegister) for IntRegister
    gpio.o(i.GPIOPortIntRegister) refers to interrupt.o(i.IntEnable) for IntEnable
    gpio.o(i.GPIOPortIntUnregister) refers to gpio.o(i.GPIOGetIntNumber) for GPIOGetIntNumber
    gpio.o(i.GPIOPortIntUnregister) refers to interrupt.o(i.IntDisable) for IntDisable
    gpio.o(i.GPIOPortIntUnregister) refers to interrupt.o(i.IntUnregister) for IntUnregister
    gpio.o(i.GPIOPinTypeComparator) refers to gpio.o(i.GPIODirModeSet) for GPIODirModeSet
    gpio.o(i.GPIOPinTypeComparator) refers to gpio.o(i.GPIOPadConfigSet) for GPIOPadConfigSet
    gpio.o(i.GPIOPinTypeI2C) refers to gpio.o(i.GPIODirModeSet) for GPIODirModeSet
    gpio.o(i.GPIOPinTypeI2C) refers to gpio.o(i.GPIOPadConfigSet) for GPIOPadConfigSet
    gpio.o(i.GPIOPinTypePWM) refers to gpio.o(i.GPIODirModeSet) for GPIODirModeSet
    gpio.o(i.GPIOPinTypePWM) refers to gpio.o(i.GPIOPadConfigSet) for GPIOPadConfigSet
    gpio.o(i.GPIOPinTypeQEI) refers to gpio.o(i.GPIODirModeSet) for GPIODirModeSet
    gpio.o(i.GPIOPinTypeQEI) refers to gpio.o(i.GPIOPadConfigSet) for GPIOPadConfigSet
    gpio.o(i.GPIOPinTypeSSI) refers to gpio.o(i.GPIODirModeSet) for GPIODirModeSet
    gpio.o(i.GPIOPinTypeSSI) refers to gpio.o(i.GPIOPadConfigSet) for GPIOPadConfigSet
    gpio.o(i.GPIOPinTypeTimer) refers to gpio.o(i.GPIODirModeSet) for GPIODirModeSet
    gpio.o(i.GPIOPinTypeTimer) refers to gpio.o(i.GPIOPadConfigSet) for GPIOPadConfigSet
    gpio.o(i.GPIOPinTypeUART) refers to gpio.o(i.GPIODirModeSet) for GPIODirModeSet
    gpio.o(i.GPIOPinTypeUART) refers to gpio.o(i.GPIOPadConfigSet) for GPIOPadConfigSet
    gpio.o(i.GPIOPinTypeCAN) refers to gpio.o(i.GPIODirModeSet) for GPIODirModeSet
    gpio.o(i.GPIOPinTypeCAN) refers to gpio.o(i.GPIOPadConfigSet) for GPIOPadConfigSet
    interrupt.o(i.IntMasterEnable) refers to cpu.o(.text) for CPUcpsie
    interrupt.o(i.IntMasterDisable) refers to cpu.o(.text) for CPUcpsid
    interrupt.o(i.IntRegister) refers to interrupt.o(vtable) for vtable
    interrupt.o(i.IntUnregister) refers to interrupt.o(i.IntDefaultHandler) for IntDefaultHandler
    interrupt.o(i.IntUnregister) refers to interrupt.o(vtable) for vtable
    interrupt.o(i.IntPriorityGroupingSet) refers to interrupt.o(.constdata) for .constdata
    interrupt.o(i.IntPriorityGroupingGet) refers to interrupt.o(.constdata) for .constdata
    interrupt.o(i.IntPrioritySet) refers to interrupt.o(.constdata) for .constdata
    interrupt.o(i.IntPriorityGet) refers to interrupt.o(.constdata) for .constdata
    ssi.o(i.SSIConfig) refers to sysctl.o(i.SysCtlClockGet) for SysCtlClockGet
    ssi.o(i.SSIIntRegister) refers to interrupt.o(i.IntRegister) for IntRegister
    ssi.o(i.SSIIntRegister) refers to interrupt.o(i.IntEnable) for IntEnable
    ssi.o(i.SSIIntUnregister) refers to interrupt.o(i.IntDisable) for IntDisable
    ssi.o(i.SSIIntUnregister) refers to interrupt.o(i.IntUnregister) for IntUnregister
    sysctl.o(i.SysCtlPeripheralPresent) refers to sysctl.o(.constdata) for .constdata
    sysctl.o(i.SysCtlPeripheralReset) refers to sysctl.o(.constdata) for .constdata
    sysctl.o(i.SysCtlPeripheralEnable) refers to sysctl.o(.constdata) for .constdata
    sysctl.o(i.SysCtlPeripheralDisable) refers to sysctl.o(.constdata) for .constdata
    sysctl.o(i.SysCtlPeripheralSleepEnable) refers to sysctl.o(.constdata) for .constdata
    sysctl.o(i.SysCtlPeripheralSleepDisable) refers to sysctl.o(.constdata) for .constdata
    sysctl.o(i.SysCtlPeripheralDeepSleepEnable) refers to sysctl.o(.constdata) for .constdata
    sysctl.o(i.SysCtlPeripheralDeepSleepDisable) refers to sysctl.o(.constdata) for .constdata
    sysctl.o(i.SysCtlIntRegister) refers to interrupt.o(i.IntRegister) for IntRegister
    sysctl.o(i.SysCtlIntRegister) refers to interrupt.o(i.IntEnable) for IntEnable
    sysctl.o(i.SysCtlIntUnregister) refers to interrupt.o(i.IntDisable) for IntDisable
    sysctl.o(i.SysCtlIntUnregister) refers to interrupt.o(i.IntUnregister) for IntUnregister
    sysctl.o(i.SysCtlSleep) refers to cpu.o(.text) for CPUwfi
    sysctl.o(i.SysCtlDeepSleep) refers to cpu.o(.text) for CPUwfi
    sysctl.o(i.SysCtlClockGet) refers to sysctl.o(.constdata) for .constdata
    timer.o(i.TimerIntRegister) refers to interrupt.o(i.IntRegister) for IntRegister
    timer.o(i.TimerIntRegister) refers to interrupt.o(i.IntEnable) for IntEnable
    timer.o(i.TimerIntUnregister) refers to interrupt.o(i.IntDisable) for IntDisable
    timer.o(i.TimerIntUnregister) refers to interrupt.o(i.IntUnregister) for IntUnregister
    timer.o(i.TimerQuiesce) refers to timer.o(i.TimerIntUnregister) for TimerIntUnregister
    stkheap2.o(.text) refers to sys_stackheap_outer.o(.text) for __user_setup_stackheap
    stkheap2.o(.text) refers to rt_stackheap_storage_intlibspace.o(.text) for __rt_stackheap_storage
    __main.o(!!!main) refers to kernel.o(.text) for __rt_entry
    kernel.o(.text) refers to stkheap2.o(.text) for __rt_stackheap_init
    kernel.o(.text) refers to boardinit2.o(.text) for _platform_post_stackheap_init
    kernel.o(.text) refers to lib_init.o(.text) for __rt_lib_init
    kernel.o(.text) refers to boardinit3.o(.text) for _platform_post_lib_init
    kernel.o(.text) refers to uart_echo.o(.text) for main
    kernel.o(.text) refers to exit.o(.text) for exit
    kernel.o(.text) refers to sys_exit.o(.text) for _sys_exit
    kernel.o(.ARM.exidx) refers to kernel.o(.text) for __rt_entry
    sys_stackheap_outer.o(.text) refers to libspace.o(.text) for __user_perproc_libspace
    sys_stackheap_outer.o(.text) refers to startup.o(.text) for __user_initial_stackheap
    rt_stackheap_storage.o(.text) refers to rt_stackheap_storage.o(.bss) for __rt_stackheap_storage_data
    rt_stackheap_storage_intlibspace.o(.text) refers (Weak) to libspace.o(.bss) for __libspace_start
    rt_stackheap_storage_onelibspace.o(.text) refers (Weak) to libspace.o(.text) for __user_libspace
    rt_stackheap_storage_twolibspace.o(.text) refers (Weak) to libspace.o(.text) for __user_perproc_libspace
    sys_exit.o(.text) refers to use_no_semi.o(.text) for __I_use_semihosting
    libspace.o(.text) refers to libspace.o(.bss) for __libspace_start
    exit.o(.text) refers to kernel.o(.text) for __rt_exit
    stkheap1.o(.text) refers to sys_stackheap_outer.o(.text) for __user_setup_stackheap
    stkheap1.o(.text) refers to rt_stackheap_storage_intlibspace.o(.text) for __rt_stackheap_storage
    lib_init.o(.emb_text) refers to no_argv.o(.text) for __ARM_get_argv
    lib_init.o(.text) refers to fpinit.o(x$fpl$fpinit) for _fp_init
    lib_init.o(.text) refers to lib_init.o(.emb_text) for __ARM_argv_veneer
    lib_init.o(.text) refers to rt_locale_intlibspace.o(.text) for __rt_locale
    rt_locale.o(.text) refers to rt_locale.o(.bss) for __rt_locale_data
    rt_locale_intlibspace.o(.text) refers (Weak) to libspace.o(.bss) for __libspace_start
    rt_locale_onelibspace.o(.text) refers (Weak) to libspace.o(.text) for __user_libspace
    rt_locale_twolibspace.o(.text) refers (Weak) to libspace.o(.text) for __user_perproc_libspace
    _get_argv.o(.text) refers to heapext.o(.text) for __heap_extend
    _get_argv.o(.text) refers to defsig_rtmem_outer.o(.text) for __rt_SIGRTMEM
    _get_argv.o(.text) refers to sys_command.o(.text) for _sys_command_string
    _get_argv.o(.text) refers (Special) to hrguard.o(.text) for __heap_region_guard
    fpinit.o(x$fpl$fpinit) refers to rt_fp_status_addr_intlibspace.o(.text) for __rt_fp_status_addr
    sys_command.o(.text) refers (Special) to use_no_semi.o(.text) for __I_use_semihosting
    rt_fp_status_addr.o(.text) refers to rt_fp_status_addr.o(.bss) for __rt_fp_status_addr_data
    rt_fp_status_addr_intlibspace.o(.text) refers (Weak) to libspace.o(.bss) for __libspace_start
    rt_fp_status_addr_onelibspace.o(.text) refers (Weak) to libspace.o(.text) for __user_libspace
    rt_fp_status_addr_twolibspace.o(.text) refers (Weak) to libspace.o(.text) for __user_perthread_libspace
    defsig_rtmem_outer.o(.text) refers to defsig_rtmem_inner.o(.text) for __rt_SIGRTMEM_inner
    defsig_rtmem_outer.o(.text) refers to defsig_exit.o(.text) for __sig_exit
    defsig_rtmem_formal.o(.text) refers to rt_raise.o(.text) for __rt_raise
    defsig_rtmem_formal.o(.text) refers (Special) to defsig_rtmem_inner.o(.text) for __rt_SIGRTMEM_inner
    heapext.o(.text) refers to stkheap2.o(.text) for __rt_heap_extend
    rt_raise.o(.text) refers to __raise.o(.text) for __raise
    rt_raise.o(.text) refers to sys_exit.o(.text) for _sys_exit
    defsig_exit.o(.text) refers to sys_exit.o(.text) for _sys_exit
    defsig_rtmem_inner.o(.text) refers to defsig_general.o(.text) for __default_signal_display
    __raise.o(.text) refers to defsig.o(CL$$defsig) for __default_signal_handler
    defsig_general.o(.text) refers to sys_wrch.o(.text) for _ttywrch
    sys_wrch.o(.text) refers (Special) to use_no_semi.o(.text) for __I_use_semihosting
    defsig.o(CL$$defsig) refers (Weak) to defsig_rtmem_inner.o(.text) for __rt_SIGRTMEM_inner


================================================================================

Removing Unused input sections from the image.

    Removing gpio.o(i.GPIOGetIntNumber), (96 bytes).
    Removing gpio.o(i.GPIODirModeGet), (38 bytes).
    Removing gpio.o(i.GPIOIntTypeSet), (56 bytes).
    Removing gpio.o(i.GPIOIntTypeGet), (50 bytes).
    Removing gpio.o(i.GPIOPadConfigGet), (122 bytes).
    Removing gpio.o(i.GPIOPinIntEnable), (12 bytes).
    Removing gpio.o(i.GPIOPinIntDisable), (12 bytes).
    Removing gpio.o(i.GPIOPinIntStatus), (14 bytes).
    Removing gpio.o(i.GPIOPinIntClear), (6 bytes).
    Removing gpio.o(i.GPIOPortIntRegister), (26 bytes).
    Removing gpio.o(i.GPIOPortIntUnregister), (22 bytes).
    Removing gpio.o(i.GPIOPinTypeComparator), (28 bytes).
    Removing gpio.o(i.GPIOPinTypeI2C), (28 bytes).
    Removing gpio.o(i.GPIOPinTypePWM), (28 bytes).
    Removing gpio.o(i.GPIOPinTypeQEI), (28 bytes).
    Removing gpio.o(i.GPIOPinTypeSSI), (28 bytes).
    Removing gpio.o(i.GPIOPinTypeTimer), (28 bytes).
    Removing gpio.o(i.GPIOPinTypeCAN), (28 bytes).
    Removing interrupt.o(i.IntMasterDisable), (4 bytes).
    Removing interrupt.o(i.IntPriorityGroupingSet), (28 bytes).
    Removing interrupt.o(i.IntPriorityGroupingGet), (36 bytes).
    Removing interrupt.o(i.IntPrioritySet), (36 bytes).
    Removing interrupt.o(i.IntPriorityGet), (24 bytes).
    Removing interrupt.o(.constdata), (92 bytes).
    Removing ssi.o(i.SSIDisable), (10 bytes).
    Removing ssi.o(i.SSIIntRegister), (32 bytes).
    Removing ssi.o(i.SSIIntUnregister), (32 bytes).
    Removing ssi.o(i.SSIIntEnable), (8 bytes).
    Removing ssi.o(i.SSIIntDisable), (8 bytes).
    Removing ssi.o(i.SSIIntStatus), (10 bytes).
    Removing ssi.o(i.SSIIntClear), (4 bytes).
    Removing ssi.o(i.SSIDataNonBlockingPut), (16 bytes).
    Removing ssi.o(i.SSIDataGet), (12 bytes).
    Removing ssi.o(i.SSIDataNonBlockingGet), (18 bytes).
    Removing sysctl.o(i.SysCtlSRAMSizeGet), (20 bytes).
    Removing sysctl.o(i.SysCtlFlashSizeGet), (20 bytes).
    Removing sysctl.o(i.SysCtlPinPresent), (20 bytes).
    Removing sysctl.o(i.SysCtlPeripheralPresent), (36 bytes).
    Removing sysctl.o(i.SysCtlPeripheralReset), (48 bytes).
    Removing sysctl.o(i.SysCtlPeripheralDisable), (28 bytes).
    Removing sysctl.o(i.SysCtlPeripheralSleepEnable), (28 bytes).
    Removing sysctl.o(i.SysCtlPeripheralSleepDisable), (28 bytes).
    Removing sysctl.o(i.SysCtlPeripheralDeepSleepEnable), (28 bytes).
    Removing sysctl.o(i.SysCtlPeripheralDeepSleepDisable), (28 bytes).
    Removing sysctl.o(i.SysCtlPeripheralClockGating), (28 bytes).
    Removing sysctl.o(i.SysCtlIntRegister), (20 bytes).
    Removing sysctl.o(i.SysCtlIntUnregister), (18 bytes).
    Removing sysctl.o(i.SysCtlIntEnable), (16 bytes).
    Removing sysctl.o(i.SysCtlIntDisable), (16 bytes).
    Removing sysctl.o(i.SysCtlIntClear), (12 bytes).
    Removing sysctl.o(i.SysCtlIntStatus), (16 bytes).
    Removing sysctl.o(i.SysCtlLDOSet), (12 bytes).
    Removing sysctl.o(i.SysCtlLDOGet), (12 bytes).
    Removing sysctl.o(i.SysCtlLDOConfigSet), (12 bytes).
    Removing sysctl.o(i.SysCtlReset), (16 bytes).
    Removing sysctl.o(i.SysCtlSleep), (4 bytes).
    Removing sysctl.o(i.SysCtlDeepSleep), (32 bytes).
    Removing sysctl.o(i.SysCtlResetCauseGet), (12 bytes).
    Removing sysctl.o(i.SysCtlResetCauseClear), (16 bytes).
    Removing sysctl.o(i.SysCtlBrownOutConfigSet), (16 bytes).
    Removing sysctl.o(i.SysCtlPWMClockSet), (20 bytes).
    Removing sysctl.o(i.SysCtlPWMClockGet), (16 bytes).
    Removing sysctl.o(i.SysCtlADCSpeedSet), (40 bytes).
    Removing sysctl.o(i.SysCtlADCSpeedGet), (16 bytes).
    Removing sysctl.o(i.SysCtlIOSCVerificationSet), (28 bytes).
    Removing sysctl.o(i.SysCtlMOSCVerificationSet), (28 bytes).
    Removing sysctl.o(i.SysCtlPLLVerificationSet), (28 bytes).
    Removing sysctl.o(i.SysCtlClkVerificationClear), (16 bytes).
    Removing timer.o(i.TimerControlLevel), (22 bytes).
    Removing timer.o(i.TimerControlTrigger), (22 bytes).
    Removing timer.o(i.TimerControlEvent), (18 bytes).
    Removing timer.o(i.TimerControlStall), (22 bytes).
    Removing timer.o(i.TimerRTCEnable), (10 bytes).
    Removing timer.o(i.TimerRTCDisable), (10 bytes).
    Removing timer.o(i.TimerPrescaleSet), (18 bytes).
    Removing timer.o(i.TimerPrescaleGet), (12 bytes).
    Removing timer.o(i.TimerPrescaleMatchSet), (18 bytes).
    Removing timer.o(i.TimerPrescaleMatchGet), (12 bytes).
    Removing timer.o(i.TimerLoadGet), (12 bytes).
    Removing timer.o(i.TimerValueGet), (12 bytes).
    Removing timer.o(i.TimerMatchGet), (12 bytes).
    Removing timer.o(i.TimerIntRegister), (92 bytes).
    Removing timer.o(i.TimerIntUnregister), (84 bytes).
    Removing timer.o(i.TimerIntEnable), (8 bytes).
    Removing timer.o(i.TimerIntDisable), (8 bytes).
    Removing timer.o(i.TimerIntStatus), (10 bytes).
    Removing timer.o(i.TimerIntClear), (4 bytes).
    Removing timer.o(i.TimerQuiesce), (58 bytes).

88 unused section(s) (total 2218 bytes) removed from the image.

================================================================================

Image Symbol Table

    Local Symbols

    Symbol Name                              Value     Ov Type        Size  Object(Section)

    RESET                                    0x00000000   Section      252  startup.o(RESET)
    ../../angel/boardlib.s                   0x00000000   Number         0  cpuinit.o ABSOLUTE
    ../../angel/boardlib.s                   0x00000000   Number         0  boardinit1.o ABSOLUTE
    ../../angel/boardlib.s                   0x00000000   Number         0  boardinit2.o ABSOLUTE
    ../../angel/boardlib.s                   0x00000000   Number         0  boardinit3.o ABSOLUTE
    ../../angel/boardlib.s                   0x00000000   Number         0  boardshut.o ABSOLUTE
    ../../angel/handlers.s                   0x00000000   Number         0  __scatter_zi.o ABSOLUTE
    ../../angel/handlers.s                   0x00000000   Number         0  __scatter_copy.o ABSOLUTE
    ../../angel/kernel.s                     0x00000000   Number         0  kernel.o ABSOLUTE
    ../../angel/rt.s                         0x00000000   Number         0  rt_stackheap_storage_onelibspace.o ABSOLUTE
    ../../angel/rt.s                         0x00000000   Number         0  rt_stackheap_storage_intlibspace.o ABSOLUTE
    ../../angel/rt.s                         0x00000000   Number         0  rt_stackheap_storage.o ABSOLUTE
    ../../angel/rt.s                         0x00000000   Number         0  rt_fp_status_addr_onelibspace.o ABSOLUTE
    ../../angel/rt.s                         0x00000000   Number         0  rt_fp_status_addr.o ABSOLUTE
    ../../angel/rt.s                         0x00000000   Number         0  rt_fp_status_addr_intlibspace.o ABSOLUTE
    ../../angel/rt.s                         0x00000000   Number         0  rt_fp_status_addr_twolibspace.o ABSOLUTE
    ../../angel/rt.s                         0x00000000   Number         0  rt_stackheap_storage_twolibspace.o ABSOLUTE
    ../../angel/rt.s                         0x00000000   Number         0  rt_locale.o ABSOLUTE
    ../../angel/rt.s                         0x00000000   Number         0  rt_locale_intlibspace.o ABSOLUTE
    ../../angel/rt.s                         0x00000000   Number         0  rt_locale_onelibspace.o ABSOLUTE
    ../../angel/rt.s                         0x00000000   Number         0  rt_raise.o ABSOLUTE
    ../../angel/rt.s                         0x00000000   Number         0  rt_locale_twolibspace.o ABSOLUTE
    ../../angel/scatter.s                    0x00000000   Number         0  __scatter.o ABSOLUTE
    ../../angel/startup.s                    0x00000000   Number         0  __main.o ABSOLUTE
    ../../angel/sys.s                        0x00000000   Number         0  sys_stackheap_outer.o ABSOLUTE
    ../../angel/sys.s                        0x00000000   Number         0  use_no_semi.o ABSOLUTE
    ../../angel/sys.s                        0x00000000   Number         0  libspace.o ABSOLUTE
    ../../angel/sys.s                        0x00000000   Number         0  sys_exit.o ABSOLUTE
    ../../angel/sysapp.c                     0x00000000   Number         0  sys_command.o ABSOLUTE
    ../../angel/sysapp.c                     0x00000000   Number         0  sys_wrch.o ABSOLUTE
    ../../armsys.c                           0x00000000   Number         0  no_argv.o ABSOLUTE
    ../../armsys.c                           0x00000000   Number         0  _get_argv.o ABSOLUTE
    ../../armsys.c                           0x00000000   Number         0  lib_init.o ABSOLUTE
    ../../armsys.c                           0x00000000   Number         0  lib_init.o ABSOLUTE
    ../../fpinit.s                           0x00000000   Number         0  fpinit.o ABSOLUTE
    ../../heapalloc.c                        0x00000000   Number         0  hrguard.o ABSOLUTE
    ../../signal.c                           0x00000000   Number         0  defsig_rtmem_formal.o ABSOLUTE
    ../../signal.c                           0x00000000   Number         0  defsig_exit.o ABSOLUTE
    ../../signal.c                           0x00000000   Number         0  defsig_rtmem_inner.o ABSOLUTE
    ../../signal.c                           0x00000000   Number         0  __raise.o ABSOLUTE
    ../../signal.c                           0x00000000   Number         0  defsig_general.o ABSOLUTE
    ../../signal.c                           0x00000000   Number         0  defsig_rtmem_outer.o ABSOLUTE
    ../../signal.s                           0x00000000   Number         0  defsig.o ABSOLUTE
    ../../stdlib.c                           0x00000000   Number         0  exit.o ABSOLUTE
    ../../stkheap.s                          0x00000000   Number         0  heapext.o ABSOLUTE
    ../../stkheap1.s                         0x00000000   Number         0  stkheap1.o ABSOLUTE
    ../../stkheap2.s                         0x00000000   Number         0  stkheap2.o ABSOLUTE
    Drivers\uart.c                           0x00000000   Number         0  uart.o ABSOLUTE
    PCD5544.c                                0x00000000   Number         0  pcd5544.o ABSOLUTE
    SRC\cpu.S                                0x00000000   Number         0  cpu.o ABSOLUTE
    SRC\gpio.c                               0x00000000   Number         0  gpio.o ABSOLUTE
    SRC\interrupt.c                          0x00000000   Number         0  interrupt.o ABSOLUTE
    SRC\ssi.c                                0x00000000   Number         0  ssi.o ABSOLUTE
    SRC\sysctl.c                             0x00000000   Number         0  sysctl.o ABSOLUTE
    SRC\timer.c                              0x00000000   Number         0  timer.o ABSOLUTE
    Startup.s                                0x00000000   Number         0  startup.o ABSOLUTE
    UART_echo.c                              0x00000000   Number         0  uart_echo.o ABSOLUTE
    dc.s                                     0x00000000   Number         0  dc.o ABSOLUTE
    NmiSR                                    0x000000f5   Thumb Code     0  startup.o(RESET)
    FaultISR                                 0x000000f7   Thumb Code     0  startup.o(RESET)
    IntDefaultHandler                        0x000000f9   Thumb Code     0  startup.o(RESET)
    !!!main                                  0x000000fc   Section        8  __main.o(!!!main)
    !!!scatter                               0x00000104   Section       52  __scatter.o(!!!scatter)
    !!handler_copy                           0x00000138   Section       26  __scatter_copy.o(!!handler_copy)
    !!handler_zi                             0x00000154   Section       28  __scatter_zi.o(!!handler_zi)
    .emb_text                                0x00000170   Section        4  lib_init.o(.emb_text)
    .text                                    0x00000174   Section       24  startup.o(.text)
    .text                                    0x0000018c   Section      508  pcd5544.o(.text)
    .text                                    0x00000388   Section      472  uart_echo.o(.text)
    .text                                    0x00000560   Section      452  uart.o(.text)
    .text                                    0x00000724   Section       12  cpu.o(.text)
    .text                                    0x00000730   Section       38  stkheap2.o(.text)
    .text                                    0x00000756   Section       62  kernel.o(.text)
    .text                                    0x00000794   Section       74  sys_stackheap_outer.o(.text)
    .text                                    0x000007e0   Section       12  rt_stackheap_storage_intlibspace.o(.text)
    .text                                    0x000007ec   Section       20  sys_exit.o(.text)
    .text                                    0x00000800   Section        8  libspace.o(.text)
    .text                                    0x00000808   Section       12  exit.o(.text)
    .text                                    0x00000814   Section      192  lib_init.o(.text)
    .text                                    0x000008d4   Section       10  boardinit2.o(.text)
    .text                                    0x000008de   Section        8  boardinit3.o(.text)
    .text                                    0x000008e6   Section        2  use_no_semi.o(.text)
    .text                                    0x000008e8   Section       12  rt_locale_intlibspace.o(.text)
    .text                                    0x000008f4   Section        2  no_argv.o(.text)
    .text                                    0x000008f8   Section       12  rt_fp_status_addr_intlibspace.o(.text)
    i.GPIODirModeSet                         0x00000904   Section       38  gpio.o(i.GPIODirModeSet)
    i.GPIOPadConfigSet                       0x0000092a   Section      148  gpio.o(i.GPIOPadConfigSet)
    i.GPIOPinRead                            0x000009be   Section        6  gpio.o(i.GPIOPinRead)
    i.GPIOPinTypeUART                        0x000009c4   Section       28  gpio.o(i.GPIOPinTypeUART)
    i.GPIOPinWrite                           0x000009e0   Section        6  gpio.o(i.GPIOPinWrite)
    i.IntDefaultHandler                      0x000009e6   Section        2  interrupt.o(i.IntDefaultHandler)
    IntDefaultHandler                        0x000009e7   Thumb Code     2  interrupt.o(i.IntDefaultHandler)
    i.IntDisable                             0x000009e8   Section       96  interrupt.o(i.IntDisable)
    i.IntEnable                              0x00000a48   Section       96  interrupt.o(i.IntEnable)
    i.IntMasterEnable                        0x00000aa8   Section        4  interrupt.o(i.IntMasterEnable)
    i.IntRegister                            0x00000aac   Section       48  interrupt.o(i.IntRegister)
    i.IntUnregister                          0x00000adc   Section       20  interrupt.o(i.IntUnregister)
    i.SSIConfig                              0x00000af0   Section       86  ssi.o(i.SSIConfig)
    i.SSIDataPut                             0x00000b46   Section       10  ssi.o(i.SSIDataPut)
    i.SSIEnable                              0x00000b50   Section       10  ssi.o(i.SSIEnable)
    i.SysCtlClockGet                         0x00000b5c   Section      156  sysctl.o(i.SysCtlClockGet)
    i.SysCtlClockSet                         0x00000bf8   Section      112  sysctl.o(i.SysCtlClockSet)
    i.SysCtlPeripheralEnable                 0x00000c68   Section       28  sysctl.o(i.SysCtlPeripheralEnable)
    i.TimerConfigure                         0x00000c84   Section       26  timer.o(i.TimerConfigure)
    i.TimerDisable                           0x00000c9e   Section       14  timer.o(i.TimerDisable)
    i.TimerEnable                            0x00000cac   Section       14  timer.o(i.TimerEnable)
    i.TimerLoadSet                           0x00000cba   Section       18  timer.o(i.TimerLoadSet)
    i.TimerMatchSet                          0x00000ccc   Section       18  timer.o(i.TimerMatchSet)
    x$fpl$fpinit                             0x00000cde   Section       14  fpinit.o(x$fpl$fpinit)
    .constdata                               0x00000cec   Section      475  pcd5544.o(.constdata)
    .constdata                               0x00000ec8   Section      112  sysctl.o(.constdata)
    g_pulDCRegs                              0x00000ec8   Data          16  sysctl.o(.constdata)
    g_pulSRCRRegs                            0x00000ed8   Data          12  sysctl.o(.constdata)
    g_pulRCGCRegs                            0x00000ee4   Data          12  sysctl.o(.constdata)
    g_pulSCGCRegs                            0x00000ef0   Data          12  sysctl.o(.constdata)
    g_pulDCGCRegs                            0x00000efc   Data          12  sysctl.o(.constdata)
    g_pulXtals                               0x00000f08   Data          48  sysctl.o(.constdata)
    vtable                                   0x20000000   Section      240  interrupt.o(vtable)
    g_pfnRAMVectors                          0x20000000   Data         240  interrupt.o(vtable)
    .bss                                     0x200000f0   Section       96  libspace.o(.bss)
    HEAP                                     0x20000150   Number         0  startup.o(HEAP)
    STACK                                    0x20000150   Section      256  startup.o(STACK)
    HeapMem                                  0x20000150   Number         0  startup.o(HEAP)
    StackMem                                 0x20000150   Data           0  startup.o(STACK)

    Global Symbols

    Symbol Name                              Value     Ov Type        Size  Object(Section)

    BuildAttributes$$THM_ISAv4$M$P$D$K$S$PE$A:L22UL41UL21$X:L11$S22US41US21$IEEE1$IW$~IW$USESV6$~STKCKD$USESV7$~SHL$OSPACE$EBA8$STANDARDLIB$REQ8$PRES8$EABIv2 0x00000000   Number         0  anon$$obj.o ABSOLUTE
    __ARM_use_no_argv                        0x00000000   Number         0  uart_echo.o ABSOLUTE
    __Vectors                                0x00000000   Data           0  startup.o(RESET)
    __ARM_exceptions_init                     - Undefined Weak Reference
    __Heap_DescSize                           - Undefined Weak Reference
    __alloca_initialize                       - Undefined Weak Reference
    __cpp_initialize__aeabi_                  - Undefined Weak Reference
    __cxa_finalize                            - Undefined Weak Reference
    __rt_SIGABRT_inner                        - Undefined Weak Reference
    __rt_SIGCPPL_inner                        - Undefined Weak Reference
    __rt_SIGFPE_inner                         - Undefined Weak Reference
    __rt_SIGILL_inner                         - Undefined Weak Reference
    __rt_SIGINT_inner                         - Undefined Weak Reference
    __rt_SIGPVFN_inner                        - Undefined Weak Reference
    __rt_SIGRTRED_inner                       - Undefined Weak Reference
    __rt_SIGSEGV_inner                        - Undefined Weak Reference
    __rt_SIGSTAK_inner                        - Undefined Weak Reference
    __rt_SIGTERM_inner                        - Undefined Weak Reference
    __rt_SIGUSR1_inner                        - Undefined Weak Reference
    __rt_SIGUSR2_inner                        - Undefined Weak Reference
    __rt_sigother_inner                       - Undefined Weak Reference
    __sigvec_lookup                           - Undefined Weak Reference
    __user_heap_extend                        - Undefined Weak Reference
    _atexit_init                              - Undefined Weak Reference
    _call_atexit_fns                          - Undefined Weak Reference
    _clock_init                               - Undefined Weak Reference
    _fp_trap_init                             - Undefined Weak Reference
    _get_lc_collate                           - Undefined Weak Reference
    _get_lc_ctype                             - Undefined Weak Reference
    _get_lc_monetary                          - Undefined Weak Reference
    _get_lc_numeric                           - Undefined Weak Reference
    _get_lc_time                              - Undefined Weak Reference
    _getenv_init                              - Undefined Weak Reference
    _handle_redirection                       - Undefined Weak Reference
    _init_alloc                               - Undefined Weak Reference
    _init_user_alloc                          - Undefined Weak Reference
    _initio                                   - Undefined Weak Reference
    _rand_init                                - Undefined Weak Reference
    _signal_init                              - Undefined Weak Reference
    _terminate_user_alloc                     - Undefined Weak Reference
    _terminateio                              - Undefined Weak Reference
    Reset_Handler                            0x000000f1   Thumb Code     0  startup.o(RESET)
    __main                                   0x000000fd   Thumb Code     8  __main.o(!!!main)
    __scatterload                            0x00000105   Thumb Code     0  __scatter.o(!!!scatter)
    __scatterload_rt2                        0x00000105   Thumb Code    44  __scatter.o(!!!scatter)
    __scatterload_rt2_thumb_only             0x00000105   Thumb Code     0  __scatter.o(!!!scatter)
    __scatterload_null                       0x00000113   Thumb Code     0  __scatter.o(!!!scatter)
    __scatterload_copy                       0x00000139   Thumb Code    26  __scatter_copy.o(!!handler_copy)
    __scatterload_zeroinit                   0x00000155   Thumb Code    28  __scatter_zi.o(!!handler_zi)
    __ARM_argv_veneer                        0x00000171   Thumb Code     4  lib_init.o(.emb_text)
    __user_initial_stackheap                 0x00000175   Thumb Code     0  startup.o(.text)
    LCD_Backlight_On                         0x0000018d   Thumb Code    56  pcd5544.o(.text)
    LCD_Backlight_Off                        0x000001c5   Thumb Code    12  pcd5544.o(.text)
    Delay                                    0x000001d1   Thumb Code    20  pcd5544.o(.text)
    LCD_Ssi_Init                             0x000001e5   Thumb Code   110  pcd5544.o(.text)
    LCD_Write                                0x00000253   Thumb Code    14  pcd5544.o(.text)
    LCD_Init                                 0x00000261   Thumb Code    60  pcd5544.o(.text)
    LCD_GotoXY                               0x0000029d   Thumb Code    44  pcd5544.o(.text)
    LCD_Cls                                  0x000002c9   Thumb Code    46  pcd5544.o(.text)
    LCD_Putchar                              0x000002f7   Thumb Code    84  pcd5544.o(.text)
    LCD_PrintStr                             0x0000034b   Thumb Code    26  pcd5544.o(.text)
    UARTIntHandler                           0x00000389   Thumb Code    50  uart_echo.o(.text)
    UARTSend                                 0x000003bb   Thumb Code    28  uart_echo.o(.text)
    main                                     0x000003d7   Thumb Code   280  uart_echo.o(.text)
    UARTParityModeSet                        0x00000561   Thumb Code    12  uart.o(.text)
    UARTParityModeGet                        0x0000056d   Thumb Code    10  uart.o(.text)
    UARTFIFOLevelSet                         0x00000577   Thumb Code     8  uart.o(.text)
    UARTFIFOLevelGet                         0x0000057f   Thumb Code    18  uart.o(.text)
    UARTEnable                               0x00000591   Thumb Code    20  uart.o(.text)
    UARTDisable                              0x000005a5   Thumb Code    30  uart.o(.text)
    UARTConfigSetExpClk                      0x000005c3   Thumb Code    48  uart.o(.text)
    UARTConfigGetExpClk                      0x000005f3   Thumb Code    30  uart.o(.text)
    UARTEnableSIR                            0x00000611   Thumb Code    22  uart.o(.text)
    UARTDisableSIR                           0x00000627   Thumb Code    10  uart.o(.text)
    UARTCharsAvail                           0x00000631   Thumb Code    12  uart.o(.text)
    UARTSpaceAvail                           0x0000063d   Thumb Code    12  uart.o(.text)
    UARTCharGetNonBlocking                   0x00000649   Thumb Code    20  uart.o(.text)
    UARTCharGet                              0x0000065d   Thumb Code    16  uart.o(.text)
    UARTCharPutNonBlocking                   0x0000066d   Thumb Code    20  uart.o(.text)
    UARTCharPut                              0x00000681   Thumb Code    14  uart.o(.text)
    UARTBreakCtl                             0x0000068f   Thumb Code    20  uart.o(.text)
    UARTIntRegister                          0x000006a3   Thumb Code    46  uart.o(.text)
    UARTIntUnregister                        0x000006d1   Thumb Code    42  uart.o(.text)
    UARTIntEnable                            0x000006fb   Thumb Code     8  uart.o(.text)
    UARTIntDisable                           0x00000703   Thumb Code     8  uart.o(.text)
    UARTIntStatus                            0x0000070b   Thumb Code    12  uart.o(.text)
    UARTIntClear                             0x00000717   Thumb Code     4  uart.o(.text)
    CPUcpsid                                 0x00000725   Thumb Code     0  cpu.o(.text)
    CPUcpsie                                 0x00000729   Thumb Code     0  cpu.o(.text)
    CPUwfi                                   0x0000072d   Thumb Code     0  cpu.o(.text)
    __use_two_region_memory                  0x00000731   Thumb Code     2  stkheap2.o(.text)
    __rt_stackheap_init                      0x00000733   Thumb Code    24  stkheap2.o(.text)
    __rt_heap_extend                         0x0000074b   Thumb Code    12  stkheap2.o(.text)
    __rt_entry                               0x00000757   Thumb Code    36  kernel.o(.text)
    __rt_exit                                0x0000077b   Thumb Code    18  kernel.o(.text)
    __rt_abort                               0x0000078d   Thumb Code     8  kernel.o(.text)
    __user_setup_stackheap                   0x00000795   Thumb Code    74  sys_stackheap_outer.o(.text)
    __rt_stackheap_storage                   0x000007e1   Thumb Code     6  rt_stackheap_storage_intlibspace.o(.text)
    _sys_exit                                0x000007ed   Thumb Code    16  sys_exit.o(.text)
    __user_libspace                          0x00000801   Thumb Code     4  libspace.o(.text)
    __user_perproc_libspace                  0x00000801   Thumb Code     0  libspace.o(.text)
    __user_perthread_libspace                0x00000801   Thumb Code     0  libspace.o(.text)
    exit                                     0x00000809   Thumb Code    12  exit.o(.text)
    __rt_lib_init                            0x00000815   Thumb Code   174  lib_init.o(.text)
    __rt_lib_shutdown                        0x000008c3   Thumb Code    18  lib_init.o(.text)
    _platform_post_stackheap_init            0x000008d5   Thumb Code    10  boardinit2.o(.text)
    _platform_post_lib_init                  0x000008df   Thumb Code     8  boardinit3.o(.text)
    __I_use_semihosting                      0x000008e7   Thumb Code     0  use_no_semi.o(.text)
    __use_no_semihosting_swi                 0x000008e7   Thumb Code     2  use_no_semi.o(.text)
    __rt_locale                              0x000008e9   Thumb Code     6  rt_locale_intlibspace.o(.text)
    __ARM_get_argv                           0x000008f5   Thumb Code     2  no_argv.o(.text)
    __rt_fp_status_addr                      0x000008f9   Thumb Code     6  rt_fp_status_addr_intlibspace.o(.text)
    GPIODirModeSet                           0x00000905   Thumb Code    38  gpio.o(i.GPIODirModeSet)
    GPIOPadConfigSet                         0x0000092b   Thumb Code   148  gpio.o(i.GPIOPadConfigSet)
    GPIOPinRead                              0x000009bf   Thumb Code     6  gpio.o(i.GPIOPinRead)
    GPIOPinTypeUART                          0x000009c5   Thumb Code    28  gpio.o(i.GPIOPinTypeUART)
    GPIOPinWrite                             0x000009e1   Thumb Code     6  gpio.o(i.GPIOPinWrite)
    IntDisable                               0x000009e9   Thumb Code    96  interrupt.o(i.IntDisable)
    IntEnable                                0x00000a49   Thumb Code    96  interrupt.o(i.IntEnable)
    IntMasterEnable                          0x00000aa9   Thumb Code     4  interrupt.o(i.IntMasterEnable)
    IntRegister                              0x00000aad   Thumb Code    42  interrupt.o(i.IntRegister)
    IntUnregister                            0x00000add   Thumb Code    10  interrupt.o(i.IntUnregister)
    SSIConfig                                0x00000af1   Thumb Code    86  ssi.o(i.SSIConfig)
    SSIDataPut                               0x00000b47   Thumb Code    10  ssi.o(i.SSIDataPut)
    SSIEnable                                0x00000b51   Thumb Code    10  ssi.o(i.SSIEnable)
    SysCtlClockGet                           0x00000b5d   Thumb Code   140  sysctl.o(i.SysCtlClockGet)
    SysCtlClockSet                           0x00000bf9   Thumb Code   108  sysctl.o(i.SysCtlClockSet)
    SysCtlPeripheralEnable                   0x00000c69   Thumb Code    24  sysctl.o(i.SysCtlPeripheralEnable)
    TimerConfigure                           0x00000c85   Thumb Code    26  timer.o(i.TimerConfigure)
    TimerDisable                             0x00000c9f   Thumb Code    14  timer.o(i.TimerDisable)
    TimerEnable                              0x00000cad   Thumb Code    14  timer.o(i.TimerEnable)
    TimerLoadSet                             0x00000cbb   Thumb Code    18  timer.o(i.TimerLoadSet)
    TimerMatchSet                            0x00000ccd   Thumb Code    18  timer.o(i.TimerMatchSet)
    _fp_init                                 0x00000cdf   Thumb Code    14  fpinit.o(x$fpl$fpinit)
    __fplib_config_pureend_doubles           0x00000ceb   Thumb Code     0  fpinit.o(x$fpl$fpinit)
    ASC2                                     0x00000cec   Data         475  pcd5544.o(.constdata)
    Region$$Table$$Base                      0x00000f38   Number         0  anon$$obj.o(Region$$Table)
    Region$$Table$$Limit                     0x00000f58   Number         0  anon$$obj.o(Region$$Table)
    __libspace_start                         0x200000f0   Data          96  libspace.o(.bss)
    __temporary_stack_top_libspace           0x20000150   Data           0  libspace.o(.bss)


================================================================================

Memory Map of the image

  Image Entry point : 0x000000fd

  Load Region LR_IROM1 (Base: 0x00000000, Size: 0x00001048, Max: 0x00002000, ABSOLUTE)

    Execution Region ER_IROM1 (Base: 0x00000000, Size: 0x00000f58, Max: 0x00002000, ABSOLUTE)

    Base Addr    Size         Type   Attr      Idx    E Section Name        Object

    0x00000000   0x000000fc   Code   RO            3    RESET               startup.o
    0x000000fc   0x00000008   Code   RO          950  * !!!main             __main.o(c_w.l)
    0x00000104   0x00000034   Code   RO         1040    !!!scatter          __scatter.o(c_w.l)
    0x00000138   0x0000001a   Code   RO         1042    !!handler_copy      __scatter_copy.o(c_w.l)
    0x00000152   0x00000002   PAD
    0x00000154   0x0000001c   Code   RO         1044    !!handler_zi        __scatter_zi.o(c_w.l)
    0x00000170   0x00000004   Code   RO          975    .emb_text           lib_init.o(c_w.l)
    0x00000174   0x00000018   Code   RO            4    .text               startup.o
    0x0000018c   0x000001fc   Code   RO           12    .text               pcd5544.o
    0x00000388   0x000001d8   Code   RO           51    .text               uart_echo.o
    0x00000560   0x000001c4   Code   RO           73    .text               uart.o
    0x00000724   0x0000000c   Code   RO          943    .text               cpu.o(DriverLib.lib)
    0x00000730   0x00000026   Code   RO          948    .text               stkheap2.o(c_w.l)
    0x00000756   0x0000003e   Code   RO          952    .text               kernel.o(c_w.l)
    0x00000794   0x0000004a   Code   RO          955    .text               sys_stackheap_outer.o(c_w.l)
    0x000007de   0x00000002   PAD
    0x000007e0   0x0000000c   Code   RO          960    .text               rt_stackheap_storage_intlibspace.o(c_w.l)
    0x000007ec   0x00000014   Code   RO          966    .text               sys_exit.o(c_w.l)
    0x00000800   0x00000008   Code   RO          968    .text               libspace.o(c_w.l)
    0x00000808   0x0000000c   Code   RO          971    .text               exit.o(c_w.l)
    0x00000814   0x000000c0   Code   RO          976    .text               lib_init.o(c_w.l)
    0x000008d4   0x0000000a   Code   RO          981    .text               boardinit2.o(c_w.l)
    0x000008de   0x00000008   Code   RO          983    .text               boardinit3.o(c_w.l)
    0x000008e6   0x00000002   Code   RO          987    .text               use_no_semi.o(c_w.l)
    0x000008e8   0x0000000c   Code   RO          992    .text               rt_locale_intlibspace.o(c_w.l)
    0x000008f4   0x00000002   Code   RO         1002    .text               no_argv.o(c_w.l)
    0x000008f6   0x00000002   PAD
    0x000008f8   0x0000000c   Code   RO         1011    .text               rt_fp_status_addr_intlibspace.o(c_w.l)
    0x00000904   0x00000026   Code   RO           93    i.GPIODirModeSet    gpio.o(DriverLib.lib)
    0x0000092a   0x00000094   Code   RO           97    i.GPIOPadConfigSet  gpio.o(DriverLib.lib)
    0x000009be   0x00000006   Code   RO          105    i.GPIOPinRead       gpio.o(DriverLib.lib)
    0x000009c4   0x0000001c   Code   RO          113    i.GPIOPinTypeUART   gpio.o(DriverLib.lib)
    0x000009e0   0x00000006   Code   RO          106    i.GPIOPinWrite      gpio.o(DriverLib.lib)
    0x000009e6   0x00000002   Code   RO          281    i.IntDefaultHandler  interrupt.o(DriverLib.lib)
    0x000009e8   0x00000060   Code   RO          291    i.IntDisable        interrupt.o(DriverLib.lib)
    0x00000a48   0x00000060   Code   RO          290    i.IntEnable         interrupt.o(DriverLib.lib)
    0x00000aa8   0x00000004   Code   RO          282    i.IntMasterEnable   interrupt.o(DriverLib.lib)
    0x00000aac   0x00000030   Code   RO          284    i.IntRegister       interrupt.o(DriverLib.lib)
    0x00000adc   0x00000014   Code   RO          285    i.IntUnregister     interrupt.o(DriverLib.lib)
    0x00000af0   0x00000056   Code   RO          376    i.SSIConfig         ssi.o(DriverLib.lib)
    0x00000b46   0x0000000a   Code   RO          385    i.SSIDataPut        ssi.o(DriverLib.lib)
    0x00000b50   0x0000000a   Code   RO          377    i.SSIEnable         ssi.o(DriverLib.lib)
    0x00000b5a   0x00000002   PAD
    0x00000b5c   0x0000009c   Code   RO          510    i.SysCtlClockGet    sysctl.o(DriverLib.lib)
    0x00000bf8   0x00000070   Code   RO          509    i.SysCtlClockSet    sysctl.o(DriverLib.lib)
    0x00000c68   0x0000001c   Code   RO          487    i.SysCtlPeripheralEnable  sysctl.o(DriverLib.lib)
    0x00000c84   0x0000001a   Code   RO          758    i.TimerConfigure    timer.o(DriverLib.lib)
    0x00000c9e   0x0000000e   Code   RO          757    i.TimerDisable      timer.o(DriverLib.lib)
    0x00000cac   0x0000000e   Code   RO          756    i.TimerEnable       timer.o(DriverLib.lib)
    0x00000cba   0x00000012   Code   RO          769    i.TimerLoadSet      timer.o(DriverLib.lib)
    0x00000ccc   0x00000012   Code   RO          772    i.TimerMatchSet     timer.o(DriverLib.lib)
    0x00000cde   0x0000000e   Code   RO         1004    x$fpl$fpinit        fpinit.o(fz_ws.l)
    0x00000cec   0x000001db   Data   RO           13    .constdata          pcd5544.o
    0x00000ec7   0x00000001   PAD
    0x00000ec8   0x00000070   Data   RO          519    .constdata          sysctl.o(DriverLib.lib)
    0x00000f38   0x00000020   Data   RO         1039    Region$$Table       anon$$obj.o


    Execution Region RW_IRAM1 (Base: 0x20000000, Size: 0x00000250, Max: 0x00000800, ABSOLUTE)

    Base Addr    Size         Type   Attr      Idx    E Section Name        Object

    0x20000000   0x000000f0   Data   RW          293    vtable              interrupt.o(DriverLib.lib)
    0x200000f0   0x00000060   Zero   RW          969    .bss                libspace.o(c_w.l)
    0x20000150   0x00000000   Zero   RW            2    HEAP                startup.o
    0x20000150   0x00000100   Zero   RW            1    STACK               startup.o


================================================================================

Image component sizes


      Code (inc. data)   RO Data    RW Data    ZI Data      Debug   Object Name

       508         36        475          0          0       7546   pcd5544.o
       276        256          0          0        256        395   startup.o
       452         10          0          0          0       4581   uart.o
       472        114          0          0          0        941   uart_echo.o

    ------------------------------------------------------------------------
      1708        416        508          0        256      13465   Object Totals
         0          0         32          0          0          0   (incl. Generated)
         0          0          1          0          0          2   (incl. Padding)

    ------------------------------------------------------------------------

      Code (inc. data)   RO Data    RW Data    ZI Data      Debug   Library Member Name

         8          0          0          0          0          0   __main.o
        52          8          0          0          0          0   __scatter.o
        26          0          0          0          0          0   __scatter_copy.o
        28          0          0          0          0          0   __scatter_zi.o
        10          0          0          0          0          0   boardinit2.o
         8          0          0          0          0          0   boardinit3.o
        12          0          0          0          0        178   cpu.o
        12          0          0          0          0          0   exit.o
        14          0          0          0          0          0   fpinit.o
       226          0          0          0          0       2740   gpio.o
       266         16          0        240          0       3216   interrupt.o
        62          0          0          0          0          0   kernel.o
       196          0          0          0          0          0   lib_init.o
         8          4          0          0         96          0   libspace.o
         2          0          0          0          0          0   no_argv.o
        12          6          0          0          0          0   rt_fp_status_addr_intlibspace.o
        12          6          0          0          0          0   rt_locale_intlibspace.o
        12          6          0          0          0          0   rt_stackheap_storage_intlibspace.o
       106          0          0          0          0       1609   ssi.o
        38          0          0          0          0          0   stkheap2.o
        20         10          0          0          0          0   sys_exit.o
        74          0          0          0          0          0   sys_stackheap_outer.o
       296         24        112          0          0       2555   sysctl.o
        90          0          0          0          0       2165   timer.o
         2          0          0          0          0          0   use_no_semi.o

    ------------------------------------------------------------------------
      1600         80        112        240         96      12463   Library Totals
         8          0          0          0          0          0   (incl. Padding)

    ------------------------------------------------------------------------

      Code (inc. data)   RO Data    RW Data    ZI Data      Debug   Library Name

       996         40        112        240          0      12463   DriverLib.lib
       582         40          0          0         96          0   c_w.l
        14          0          0          0          0          0   fz_ws.l

    ------------------------------------------------------------------------
      1600         80        112        240         96      12463   Library Totals

    ------------------------------------------------------------------------

================================================================================


      Code (inc. data)   RO Data    RW Data    ZI Data      Debug   

      3308        496        620        240        352      25928   Grand Totals
      3308        496        620        240        352      25928   ELF Image Totals
      3308        496        620        240          0          0   ROM Totals

================================================================================

    Total RO  Size (Code + RO Data)                 3928 (   3.84kB)
    Total RW  Size (RW Data + ZI Data)               592 (   0.58kB)
    Total ROM Size (Code + RO Data + RW Data)       4168 (   4.07kB)

================================================================================

